:020000040800F2
:1000000000000120513D0008493800084B38000825
:100010004D3800084F380008513800080000000033
:10002000000000000000000000000000E1280008BF
:10003000533800080000000081290008E529000865
:10004000A13D0008A13D0008A13D0008A13D000818
:10005000A13D0008A13D0008A13D0008A13D000808
:10006000A13D0008A13D0008A13D0008A13D0008F8
:10007000A13D0008A13D0008A13D0008A13D0008E8
:10008000A13D0008A13D0008A13D000800000000BE
:10009000000000000000000000000000A13D00087A
:1000A000A13D0008A13D0008A13D0008A13D0008B8
:1000B000A13D0008A13D0008A13D0008A13D0008A8
:1000C000A13D0008A13D0008A13D0008A13D000898
:1000D000A13D0008A13D0008A13D0008000000006E
:1000E000A13D0008A13D0008A13D0008000000005E
:1000F000000000000000000000000000A13D00081A
:1001000000000000A13D000855380008A13D00088E
:1001100000000000000000000000000000000000DF
:10012000A13D0008A13D0008A13D0008A13D000837
:10013000A13D0008000000000000000000000000D9
:10014000000000000000000000000000A13D0008C9
:10015000A13D0008A13D0008A13D0008A13D000807
:10016000A13D0008A13D00080000000000000000C3
:10017000000000000000000000000000000000007F
:1001800000000000A13D0008000000000000000089
:04019000A13D000885
:1001A00010B5054C237833B9044B13B10448AFF3B1
:1001B00000800123237010BDD00300200000000048
:1001C000FC3D000808B5034B1BB103490348AFF3DE
:1001D000008008BD00000000D4030020FC3D0008A2
:1001E00053B94AB9002908BF00281CBF4FF0FF319E
:1001F0004FF0FF3000F072B9ADF1080C6DE904CE9C
:1002000000F006F8DDF804E0DDE9022304B07047F1
:100210002DE9F047089E04468846002B4BD18A42C0
:10022000154667D9B2FA82F24AB1C2F1200701FA43
:1002300002F320FA07F7954047EA030894404FEA93
:10024000154E230CB8FBFEF71FFA85FC0EFB178832
:1002500043EA084307FB0CF1994209D9EB1807F16F
:10026000FF3080F01B81994240F21881023F2B44FD
:100270005B1AA4B2B3FBFEF00EFB103344EA034456
:1002800000FB0CFCA44509D92C1900F1FF3380F0C8
:100290000781A44540F2048102382C4440EA07401B
:1002A000A4EB0C0400271EB1D4400023C6E9004390
:1002B0003946BDE8F0878B4209D9002E00F0EB806B
:1002C0000027C6E9000138463946BDE8F087B3FA91
:1002D00083F7002F47D18B4202D3824200F2FA808B
:1002E000841A61EB030301209846002EE0D0C6E992
:1002F0000048DDE702B9FFDEB2FA82F2002A40F0E0
:100300008F80491B4FEA154E1FFA85F80127B1FB74
:10031000FEFC230C0EFB1C1143EA014308FB0CF10D
:10032000994207D9EB180CF1FF3002D2994200F242
:10033000CD808446591AA3B2B1FBFEF00EFB101417
:1003400043EA044408FB00F8A04507D92C1900F142
:10035000FF3302D2A04500F2B6801846A4EB080491
:1003600040EA0C409FE7C7F1200CBB4022FA0CFE8C
:100370004EEA030E01FA07F420FA0CF521FA0CF309
:100380004FEA1E482543B3FBF8F92C0C08FB193340
:100390001FFA8EFA44EA034309FB0AF49C4202FA6C
:1003A00007F200FA07F10BD91EEB030309F1FF3046
:1003B00080F087809C4240F28480A9F10209734456
:1003C0001B1BADB2B3FBF8F008FB103345EA034446
:1003D00000FB0AFAA24508D91EEB040400F1FF3322
:1003E0006BD2A24569D90238744440EA0940A0FBA7
:1003F0000289A4EB0A044C45C2464B4654D351D063
:10040000002E69D0B1EB0A0564EB030404FA0CFC7E
:10041000FD40FC404CEA0505C6E90054002747E7CB
:10042000C2F1200320FA03F7954001FA02F021FA05
:1004300003F34FEA154E3843010CB3FBFEF71FFAE6
:1004400085F80EFB173341EA034107FB08F38B42A3
:1004500004FA02F407D9691807F1FF3C2FD28B4246
:100460002DD9023F2944CB1A81B2B3FBFEF00EFB1B
:10047000103341EA034100FB08F38B4207D96918A6
:1004800000F1FF3C17D28B4215D902382944C91A12
:1004900040EA07473BE73746304609E70746E7E6C5
:1004A0001846FBE64145ABD2B8EB020A69EB0E02F7
:1004B00001381346A4E76046E9E7184695E7674622
:1004C000D1E781467CE702382C4447E7ACF1020CC7
:1004D0002B442FE7384608E73746E9E6704700BF68
:1004E00008B50B4B1A6842F400721A601A6842F49D
:1004F00080621A601A6842F480721A60032000F069
:10050000A5F9002003F062F903F03EF9002008BDD0
:10051000003C0240034A1168034B1B780B441360F4
:10052000704700BF3C41002000000020014B1868CC
:10053000704700BF3C410020494B5A6822F44032CA
:100540005A605A6841680A435A600268536823F443
:100550008073536002685368016943EA0123536062
:100560000268536823F040735360026853688168DF
:100570000B4353600268936823F40063936002683E
:100580009368C1680B439360826A364B9A4249D0A4
:100590000268936823F07063936002689368816ACD
:1005A0000B4393600268936823F0405393600268A2
:1005B0009368C16A0B4393600268936823F0020357
:1005C000936002689368816943EA41039360036A18
:1005D000002B32D10268536823F400635360026831
:1005E000D36A23F47003D3620168CB6AC269013A0B
:1005F00043EA0253CB620268936823F4007393606A
:1006000002689368016B43EA412393600268936830
:1006100023F48063936002689368416943EA81230D
:10062000936070470268936823F070639360026878
:10063000936823F040539360BEE70268536843F425
:10064000006353600268536823F460435360016899
:100650004B68426A013A43EA42334B60BFE700BF4E
:10066000002301400100000F30B310B50446036CB5
:1006700043B1236C13F0100F0AD00120002384F83B
:100680003C3010BD436480F83C3002F03FFDF0E7A1
:10069000236C23F4885323F0020343F00203236402
:1006A0002046FFF749FF00206064236C23F003031A
:1006B00043F001032364E1E70120704730B482B0C6
:1006C0000023019390F83C30012B00F0B780012308
:1006D00080F83C300B68092B3ED90568EA689BB26C
:1006E00003EB43031E3B072404FA03F322EA03034C
:1006F000EB600568EA688C680B8803EB43031E3BDC
:1007000004FA03F31343EB604B68062B3AD80568F1
:100710006A6B03EB8303053B1F2404FA03F322EA0D
:1007200003036B6305686A6B4B6803EB8303053B4C
:100730000C8804FA03F313436B630268404B9A423C
:1007400050D002683E4B9A4255D0002380F83C308E
:10075000184602B030BC704705682A699BB203EBAB
:100760004303072404FA03F322EA03032B61056819
:100770002A698C680B8803EB430304FA03F31343E1
:100780002B61C1E70C2B16D805682A6B03EB83039A
:10079000233B1F2404FA03F322EA03032B630568B7
:1007A0002A6B4B6803EB8303233B0C8804FA03F3A7
:1007B00013432B63C1E70568EA6A03EB8303413BFC
:1007C0001F2404FA03F322EA0303EB620568EA6AD2
:1007D0004B6803EB8303413B0C8804FA03F3134398
:1007E000EB62AAE70B68122BABD1164A536843F4AD
:1007F00080035360A5E70B68103B012BA5D8114A75
:10080000536843F4000353600B68102B9DD10E4BCB
:100810001B6802F1467202F52E3202F28332A2FB0D
:1008200003239B0C03EB83035A00019202E0019B1C
:10083000013B0193019B002BF9D186E7022088E759
:100840000020014000230140CC030020074AD36868
:1008500023F4E0631B041B0C000200F4E060184367
:1008600040F0BF6040F40030D060704700ED00E021
:1008700030B4174BDB68C3F30223C3F10704042C25
:1008800028BF04241D1D062D18D9033B4FF0FF354A
:1008900005FA04F421EA0401994005FA03F322EA77
:1008A0000303194300280BDB0901C9B200F16040C2
:1008B00000F5614080F8001330BC70470023E5E785
:1008C00000F00F000901C9B2024B1954F4E700BF50
:1008D00000ED00E014ED00E000F01F0240090123EC
:1008E0009340024A42F82030704700BF00E100E028
:1008F00000230F2B00F2C580F0B482B039E004224F
:1009000000E00022B2403A4302345E4E46F8242012
:100910005D4A1468EA4302EA04064F6817F4803F10
:1009200001D045EA0406584C2660646802EA0406D1
:100930004F6817F4003F01D045EA0406524C666048
:10094000A46802EA04064F6817F4801F01D045EA44
:1009500004064D4CA660E46822404E6816F4001F61
:1009600001D045EA0402484CE26001330F2B00F24B
:10097000858001229A400C6804EA0205AA42F4D15B
:100980004C68022C01D0122C10D1DE08083650F829
:1009900026C003F00704A7000F24BC402CEA040C77
:1009A0000C69BC4044EA0C0440F8264004685F002F
:1009B0000326BE40F64306EA040C4C6804F0030428
:1009C000BC4044EA0C0404604C6804F1FF3CBCF1F8
:1009D000010F03D9112C01D0122C10D1846806EA22
:1009E000040CCC68BC4044EA0C048460446824EAEB
:1009F00002024C68C4F300149C4014434460C26873
:100A000016408A68BA403243C2604A6812F0805F7A
:100A1000ABD0002201921D4A546C44F480445464CB
:100A2000526C02F480420192019A9C08A61C154A5D
:100A300052F8267003F0030296000F22B24027EA14
:100A40000207134A90423FF45CAF02F58062904285
:100A50000ED002F5806290420CD002F58062904286
:100A60000AD002F5806290423FF449AF072249E77D
:100A7000012247E7022245E7032243E702B0F0BC28
:100A80007047704700380140003C01400038024088
:100A90000000024012B9090481617047816170470A
:100AA00003685A6912F4806F0DD06FF480625A6146
:100AB0000423036400230363202280F83D2080F890
:100AC0003C300120704700207047F8B506460C46C0
:100AD00017461D461EE02DB1FFF728FD069BC01AE4
:100AE000A84217D900233363202286F83D2086F8D8
:100AF0003E3086F83C3003201AE033685B6924EA14
:100B000003039BB2B3FA83F35B099F420FD1B5F1A4
:100B1000FF3FE0D1C4F30743012BEED033689B695C
:100B200024EA03039BB2B3FA83F35B09EDE70020E9
:100B3000F8BDF8B504460D4616461F4632E01A6861
:100B400042F400721A6023686FF480625A610423D1
:100B5000236400232363202284F83D2084F83C3062
:100B600001202DE026B1FFF7E1FCC01BB04219D9EE
:100B700000232363202284F83D2084F83C300320A6
:100B80001EE023685B6925EA03039BB2003318BFAC
:100B90000123A3B123685A6912F4806FCFD1B6F153
:100BA000FF3FDFD1C5F30743012BEAD023689B69E0
:100BB00025EA03039BB2003318BF0123E9E70020B5
:100BC000F8BD0000F0B583B004460D4616461F463A
:100BD000C36A042B0DD0012B0BD013F5803F08D036
:100BE000036B122B0AD10268136843F480731360FD
:100BF00004E02268136843F480731360009733465F
:100C000000224FF001112046FFF75FFF58BB236918
:100C1000B3F5804F10D1236805F0FE051D613B46FA
:100C2000324615492046FFF784FF0346E0B1236CA6
:100C3000042B1ED1012317E0EB11226803F00603F9
:100C400043F0F00313613B4632460C492046FFF760
:100C500070FF20B1236C042B09D1012304E0236829
:100C6000EDB21D61DBE70323184603B0F0BD03239B
:100C7000FAE70323F8E700BF0200010008000100C3
:100C80002DE9F04184B004460D4616461F46C26A5F
:100C900001680B6843F480630B60042A0DD0012ABD
:100CA0000BD012F5803F08D0036B112B0AD10268DC
:100CB000136843F48073136004E02268136843F4FC
:100CC000807313600097334600224FF001112046D5
:100CD000FFF7FBFE002852D12369B3F5804F12D1F4
:100CE000236845F00105EDB21D613B4632462A49B5
:100CF0002046FFF71EFF0346002841D0236C042B3B
:100D000048D101233CE04FEAE51808F006082368C3
:100D100048F0F0021A613B46324620492046FFF770
:100D200008FF20B1236C042B2ED1012328E0236877
:100D3000EDB21D613B46324617492046FFF7F9FEEA
:100D400020B1236C042B21D1012319E0002203924E
:100D5000236859690391996903910399196841F4CA
:100D600080711960009733464FF001112046FFF75C
:100D7000ACFE68B9226848F0F1031361B5E70323BC
:100D8000184604B0BDE8F0810323F9E70323F7E731
:100D90000323F5E70323F3E7020001000800010045
:100DA00070B504460D46164623685B6913F0800F44
:100DB00019D12046FFF774FEB8B9B5F1FF3FF3D063
:100DC00025B1FFF7B3FB801BA842EDD9236C43F09C
:100DD0002003236400232363202284F83D2084F829
:100DE0003C30032000E0002070BD0120FCE770B51E
:100DF00004460D46164623685B6913F0040F19D1AB
:100E00002046FFF74DFEB8B9B5F1FF3FF3D025B14D
:100E1000FFF78CFB801BA842EDD9236C43F0200325
:100E2000236400232363202284F83D2084F83C308F
:100E3000032000E0002070BD0120FCE770B50546EE
:100E40000C4616462B685A6912F0400F22D15A6997
:100E500012F0100F11D124B1FFF768FB801BA042E4
:100E6000F0D92B6C43F020032B64202385F83D3010
:100E7000002385F83C30032070BD6FF010025A61EA
:100E800000232B642B63202285F83D2085F83C301D
:100E90000120F1E70020EFE7002800F0828010B584
:100EA000044690F83D30002B41D0242384F83D3097
:100EB0002268136823F00103136000F083FD3A4BAE
:100EC000A3FB00239B0C226853606168374A914260
:100ED00032D80133226813626368344A934235D8AA
:100EE0005B00B0FBF3F0C0F30B03032B00D804202E
:100EF0002368D861E369216A22680B431360236980
:100F0000E16822680B4393606369A16922680B431F
:100F1000D3602268136843F001031360002020644B
:100F2000202384F83D30206384F83E0010BD80F813
:100F30003C3002F0B9FAB8E74FF4967202FB03F3C3
:100F40001B4AA2FB03239B090133C3E7A16889B9AC
:100F500003EB4302B0FBF2F2C2F30B02B2FA82F2ED
:100F60005209E2B991B903EB4303B0FBF3F040F44B
:100F70000040BDE703EB830202EB8202B0FBF2F21A
:100F8000C2F30B02B2FA82F25209EAE703EB8303DF
:100F900003EB8303B0FBF3F040F44040A8E70120EB
:100FA000A6E70120704700BF83DE1B43A086010037
:100FB000D34D62102DE9F04184B004460E469046B0
:100FC0001F46FFF7B3FA94F83D30DBB2202B04D074
:100FD0000226304604B0BDE8F08105460090192392
:100FE000012254492046FFF770FD002840F0998007
:100FF00094F83C30012B00F09680012384F83C30BB
:1010000023681A6812F0010F03D11A6842F0010236
:101010001A602268136823F400631360212384F8A4
:101020003D30102384F83E3000232364C4F824802C
:101030006785A3F58033E362638D23852B460A9A87
:1010400031462046FFF7BEFD064660B1236C042BF7
:1010500004D1002384F83C300126BAE7002384F849
:101060003C300326B5E70023039323685A690392B3
:101070009B690393039B10E0236C042B55D12268DA
:10108000136843F4007313600126A2E72A460A9905
:101090002046FFF7ACFE00282BD1238D002B32D049
:1010A0002A460A992046FFF77BFE0028E4D1636AAE
:1010B0005A1C626222681B781361638D013B9BB2EC
:1010C0006385238D013B9BB223852268516911F012
:1010D000040FDBD0002BD9D0636A591C61621B78E6
:1010E0001361638D013B9BB26385238D013B238597
:1010F000CCE7236C042B1AD12268136843F40073E5
:101100001360012665E72268136843F400731360D7
:10111000202384F83D30002384F83E3084F83C30AE
:1011200057E7022655E7022653E7032651E7032631
:101130004FE700BF020010002DE9F04186B00446E1
:101140000E4690461F46FFF7F1F994F83D30DBB2AA
:10115000202B04D00226304606B0BDE8F0810546BB
:101160000090192301228C492046FFF7AEFC00288D
:1011700040F04B8194F83C30012B00F04881012372
:1011800084F83C3023681A6812F0010F03D11A6802
:1011900042F001021A602268136823F400631360AE
:1011A000222384F83D30102384F83E30002323644A
:1011B000C4F824806785A3F58033E362638D2385BB
:1011C0002B460C9A31462046FFF75AFD064660B181
:1011D000236C042B04D1002384F83C300126BAE7A9
:1011E000002384F83C300326B5E7238D5BB90293D6
:1011F00023685A6902929A690292029A1A6842F422
:1012000000721A607AE0012B0FD0022B1FD02268E7
:10121000136843F4806313600023059323685A69BD
:1012200005929B690593059B68E02268136823F487
:10123000806313600023039323685A6903929A69B9
:101240000392039A1A6842F400721A6056E0226808
:10125000136823F4806313602268136843F4006307
:1012600013600023049323685A6904929B690493D2
:10127000049B43E02A460C992046FFF7DFFD68B93E
:1012800023681A69636A591C61621A70238D013BD5
:101290002385638D013B9BB263852FE0236C202B5C
:1012A00001D0012657E7032655E700950C9B002245
:1012B0003A492046FFF709FC002840F0AA8022683E
:1012C000136843F40073136023681A69636A591C36
:1012D00061621A70238D013B2385638D013B9BB2B4
:1012E000638523681A69636A591C61621A70238DC9
:1012F000013B2385638D013B9BB26385238D002BCE
:101300007AD0032B4CD8012BB4D0022BCDD0009532
:101310000C9B002221492046FFF7D7FB00287AD1F9
:101320002268136823F48063136023681A69636A70
:10133000591C61621A70238D013B2385638D013B2B
:101340009BB2638500950C9B002214492046FFF751
:10135000BCFB002861D12268136843F4007313605A
:1013600023681A69636A591C61621A70238D013BF4
:101370002385638D013B9BB2638523681A69636A89
:10138000591C61621A70238D013B2385638D013BDB
:101390009BB26385B2E700BF0200100004000100A9
:1013A0002A460C992046FFF749FDF0B923681A69CF
:1013B000636A591C61621A70238D013B2385638D1A
:1013C000013B9BB2638523685A6912F0040F95D0E4
:1013D0001A69636A591C61621A70238D013B238567
:1013E000638D013B9BB2638588E7236C202B01D082
:1013F0000126B0E60326AEE6202384F83D30002324
:1014000084F83E3084F83C30A5E60226A3E60226A6
:10141000A1E603269FE603269DE603269BE600BF82
:10142000002800F0BB8170B582B00446036813F059
:10143000010F3BD0A74B9B6803F00C03042B2CD06F
:10144000A44B9B6803F00C03082B21D06368B3F511
:10145000803F4FD0B3F5A02F52D09E4B1A6822F494
:1014600080321A601A6822F480221A606368002BA6
:1014700050D0FFF75BF80546964B1B6813F4003F0E
:1014800014D1FFF753F8401B6428F5D903208AE1F3
:10149000904B5B6813F4800FD8D08E4B1B6813F40D
:1014A000003F03D06368002B00F07A81236813F0BB
:1014B000020F55D0874B9B6813F00C0F3ED0854B25
:1014C0009B6803F00C03082B33D0E368002B68D033
:1014D000814B01221A60FFF729F805467D4B1B68F6
:1014E00013F0020F54D1FFF721F8401B0228F5D961
:1014F000032058E1774A136843F480331360B5E75B
:10150000744B1A6842F480221A601A6842F48032DE
:101510001A60ABE7FFF70AF805466E4B1B6813F439
:10152000003FC3D0FFF702F8401B6428F5D9032021
:1015300039E1684B5B6813F4800FC6D1654B1B68BB
:1015400013F0020F04D0E368012B01D001202AE13F
:10155000604A136823F0F803216943EAC10313606A
:10156000236813F0080F40D0636963B35B4B01221B
:101570001A60FEF7DBFF0546564B5B6F13F0020F58
:1015800033D1FEF7D3FF401B0228F5D903200AE12F
:10159000504A136823F0F803216943EAC10313603A
:1015A000DEE74D4B00221A60FEF7C0FF0546494BAF
:1015B0001B6813F0020FD3D0FEF7B8FF401B0228C0
:1015C000F5D90320EFE0454B00221A60FEF7AEFF8D
:1015D0000546404B5B6F13F0020F06D0FEF7A6FFE7
:1015E000401B0228F5D90320DDE0236813F0040F27
:1015F00079D0384B1B6C13F0805F33D100230193FB
:10160000344B1A6C42F080521A641B6C03F0805306
:101610000193019B0125324B1B6813F4807F23D07B
:10162000A368012B34D0052B38D02A4B1A6F22F037
:1016300001021A671A6F22F004021A67A368002BCE
:1016400036D0FEF773FF0646224B1B6F13F0020FD6
:1016500048D1FEF76BFF801B41F288339842F3D9E3
:101660000320A0E00025D6E71D4A136843F48073E9
:101670001360FEF75BFF0646194B1B6813F4807F6F
:10168000CED1FEF753FF801B0228F5D903208AE054
:10169000104A136F43F001031367CFE70D4B1A6F26
:1016A00042F004021A671A6F42F001021A67C5E796
:1016B000FEF73CFF0646074B1B6F13F0020F11D0DD
:1016C000FEF734FF801B41F288339842F3D90320A0
:1016D00069E000BF0038024000004742800E4742E8
:1016E00000700040E5B9A369002B5BD0304A9268D6
:1016F00002F00C02082A58D0022B17D02D4B0022E2
:101700001A60FEF713FF0446294B1B6813F0007F95
:1017100042D0FEF70BFF001B0228F5D9032042E060
:10172000234A136C23F080531364DCE7214B00221F
:101730001A60FEF7FBFE05461D4B1B6813F0007F89
:1017400006D0FEF7F3FE401B0228F5D903202AE05D
:10175000E369226A1343626A43EA8213A26A520867
:10176000013A43EA0243E26A43EA0263104A5360E1
:10177000104B01221A60FEF7D9FE04460C4B1B6881
:1017800013F0007F06D1FEF7D1FE001B0228F5D929
:10179000032008E0002006E0002004E0012070475C
:1017A000012000E0002002B070BD0120FBE700BF77
:1017B0000038024060004742264B9B6803F00C0350
:1017C000042B44D0082B01D0234870472DE9F04B5F
:1017D000204B5A6802F03F025B6813F4800F13D06D
:1017E0001C4B5968C1F3881100231C48A1FB000160
:1017F000FEF7F6FC174B5B68C3F3014301335B0054
:10180000B0FBF3F0BDE8F08B124B5B68C3F38813B9
:101810001E4600275C010025E41A65EB0705A901B7
:1018200041EA9461A001001B61EB0501CB0043EA92
:101830005073C400A01943EB07018B0243EA905395
:101840008402204619460023FEF7CAFCD2E703486B
:10185000704700BF003802400024F40040787D014A
:10186000002800F09D8070B504464F4B1B6803F0C4
:101870000F038B4209D2CBB24B4A1370136803F0AB
:101880000F038B4201D0012070BD236813F0020FBB
:1018900017D013F0040F04D0444A936843F4E05384
:1018A0009360236813F0080F04D0404A936843F410
:1018B000604393603D4A936823F0F003A0680343BC
:1018C00093600D46236813F0010F32D06368012B3B
:1018D00021D09A1E012A25D9344A126812F0020F2B
:1018E00060D032498A6822F0030213438B60FEF70E
:1018F0001DFE06462D4B9B6803F00C036268B3EB9C
:10190000820F16D0FEF712FE801B41F288339842F8
:10191000F0D90320B8E7254A126812F4003FE0D15D
:101920000120B1E7214A126812F0007FD9D10120CD
:10193000AAE71D4B1B6803F00F03AB4209D9EAB2BB
:10194000194B1A701B6803F00F03AB4201D0012042
:101950009AE7236813F0040F06D0144A936823F41F
:10196000E053E1680B439360236813F0080F07D03E
:101970000E4A936823F46043216943EAC1039360EC
:10198000FFF71AFF094B9B68C3F30313084AD35CA4
:10199000D840084B1860002001F018FF002073E7C2
:1019A0000120704701206FE7003C024000380240F0
:1019B000283E0008CC030020014B1868704700BF88
:1019C000CC03002008B5FFF7F7FF044B9B68C3F377
:1019D0008223034AD35CD84008BD00BF00380240D0
:1019E000383E00080F2303600B4B9A6802F0030295
:1019F00042609A6802F0F00282609A6802F4E05253
:101A0000C2609B68DB0803F4E0530361034B1B686F
:101A100003F00F030B60704700380240003C0240A7
:101A200000283BD010B504460023836290F8513063
:101A3000002B2ED0022384F851302268136823F043
:101A4000400313606368A2681343E268134322698A
:101A5000134362691343A26902F400721343E269FB
:101A60001343226A1343A16A22680B431360638BFA
:101A700003F00403616A22680B4353602268D36950
:101A800023F40063D36100206065012384F85130A2
:101A900010BD80F8503001F03FFECBE701207047C9
:101AA00070B4036A23F001030362036A4268846925
:101AB00024F073040D6845EA040623F002048B68E1
:101AC00023430B4DA84206D0426086614A684263B8
:101AD000036270BC704723F00803CC68234323F0F3
:101AE000040322F440724C6914438A692243EBE7F1
:101AF0000000014030B4036A23F480730362036A78
:101B00004268C46924F073040D682C4323F4007305
:101B10008D6843EA05230D4DA84206D04260C4619A
:101B20004A68C263036230BC704723F40063CD6827
:101B300043EA052323F4806322F440524D6942EACC
:101B400005128D6942EA0512E8E700BF0000014076
:101B500030B4036A23F480530362036A4468C269A1
:101B600022F4E6420D6842EA052223F400538D6810
:101B700043EA0533074DA84206D04460C2614A6873
:101B80000264036230BC704724F480444D6944EA27
:101B90008514F2E70000014010B4036A046A24F0DF
:101BA00001040462846924F0F00444EA021223F080
:101BB0000A030B43826103625DF8044B704710B463
:101BC000036A23F0100303628469036A24F47044F7
:101BD00044EA023223F0A00343EA01138261036264
:101BE0005DF8044B704710B4846824F47F4442EAE3
:101BF00003230B43234383605DF8044B704710B508
:101C00000468A26822F070024B68134323F00703B4
:101C10000A681343A3604B68502B1ED00AD9602B6F
:101C200021D0702B05D10B698A68C9680068FFF75D
:101C3000DAFF10BD402BFCD103681C6A1A6A22F03F
:101C400001021A620268936923F0F003096943EA0A
:101C50000113936103681C62EBE70A6989680068F5
:101C6000FFF79AFFE5E70A6989680068FFF7A7FFB1
:101C7000DFE70268D36843F00103D36002681368AA
:101C800043F0010313600020704738B590F83830F6
:101C9000012B18D00446012580F83850022380F823
:101CA0003930FFF7ACFF2268D36823F04003D360DC
:101CB0002268D36823F48043D36084F8395000202D
:101CC00084F8380038BD0220FCE770477047704741
:101CD000704710B5044603681A6912F0020F11D05C
:101CE000DA6812F0020F0DD06FF002021A610123C0
:101CF000037603689B6913F0030F70D0FFF7E6FFCC
:101D00000023237623681A6912F0040F12D0DA68D0
:101D100012F0040F0ED06FF004021A610223237632
:101D200023689B6913F4407F5FD02046FFF7CEFF06
:101D30000023237623681A6912F0080F12D0DA689C
:101D400012F0080F0ED06FF008021A6104232376F8
:101D50002368DB6913F0030F4ED02046FFF7B6FF70
:101D60000023237623681A6912F0100F12D0DA6864
:101D700012F0100F0ED06FF010021A6108232376B4
:101D80002368DB6913F4407F3DD02046FFF79EFFB8
:101D90000023237623681A6912F0010F03D0DA6852
:101DA00012F0010F36D123681A6912F0800F03D0A8
:101DB000DA6812F0800F34D123681A6912F0400FEC
:101DC00003D0DA6812F0400F32D123681A6912F09A
:101DD000200F03D0DA6812F0200F30D110BDFFF7CA
:101DE00074FF2046FFF773FF8AE72046FFF76DFF79
:101DF0002046FFF76CFF9BE72046FFF766FF204673
:101E0000FFF765FFACE72046FFF75FFF2046FFF7CF
:101E10005EFFBDE76FF001021A61204601F0D8FBBA
:101E2000C1E76FF080021A61204600F051F9C3E764
:101E30006FF040021A612046FFF74AFFC5E76FF0D6
:101E400020021A61204600F042F9C7E70368234ADE
:101E500090420ED0B0F1804F0BD0A2F57C42904260
:101E600007D002F58062904203D002F58062904272
:101E700003D123F070034A681343184A90421AD0E2
:101E8000B0F1804F17D0A2F57C42904213D002F5FA
:101E9000806290420FD002F5806290420BD002F532
:101EA0009A32904207D002F58062904203D002F548
:101EB0008062904203D123F44073CA6813430360E5
:101EC0008B68C3620B688362044B984202D0012383
:101ED000436170470B690363F9E700BF00000140ED
:101EE000A8B110B5044690F839305BB1022384F8EC
:101EF0003930211D2068FFF7A9FF012384F839300C
:101F0000002010BD80F8383001F04CFDEEE70120D4
:101F10007047A8B110B5044690F839305BB1022380
:101F200084F83930211D2068FFF790FF012384F8E1
:101F30003930002010BD80F8383001F05DFDEEE74B
:101F40000120704730B4036A23F010030362036A70
:101F50004468826922F4E6420D6842EA052223F0D1
:101F600020038D6843EA05130C4DA84206D0446057
:101F700082614A688263036230BC704723F0800349
:101F8000CD6843EA051323F0400324F440644D690F
:101F900044EA85048D6944EA8504E8E700000140CD
:101FA00038B590F83830012B66D00D460446012331
:101FB00080F83830022380F839300C2A1AD8DFE84C
:101FC00002F007191919201919193419191947009C
:101FD0000068FFF765FD2268936943F00803936189
:101FE0002268936923F00403936122689369296945
:101FF0000B439361012384F83930002084F83800C2
:1020000038BD0068FFF79EFF2268936943F40063C0
:1020100093612268936923F48063936122689369D2
:10202000296943EA01239361E4E70068FFF762FD51
:102030002268D36943F00803D3612268D36923F08F
:102040000403D3612268D36929690B43D361D1E7C3
:102050000068FFF77DFD2268D36943F40063D36114
:102060002268D36923F48063D3612268D369296924
:1020700043EA0123D361BDE70220C1E790F838307D
:10208000012B22D030B4012280F83820022380F8BE
:1020900039300468636823F0700363600468636820
:1020A0000D682B4363600468A36823F08003A3607A
:1020B0000468A36849680B43A36080F839200023B3
:1020C00080F83830184630BC70470220704770479F
:1020D0007047842801D0033070470020704708B54E
:1020E00000F0C0F9002008BDF0B585B00F46446887
:1020F00005680669B0F90800FFF7EBFF03AB019331
:1021000000903B46B2B22946204600F079F90128FA
:1021100002D1039805B0F0BD0020FBE708B50346E7
:1021200000B90123184600F0DFFA002008BD00F1D5
:10213000080343604FF0FF328260C36003610023F5
:102140000360704700230361704743684B609A68DF
:102150008A609A685160996008610368013303607E
:10216000704730B40D68B5F1FF3F02D000F10802AE
:1021700002E0026904E01A4653681C68AC42FAD9CE
:1021800053684B6099608A6051600861036801334D
:10219000036030BC7047036942688168916082685F
:1021A000416851605A68824205D000220261186875
:1021B00001381860704782685A60F6E7074B9B6ADF
:1021C0001B6833B1054B9A6AD268D2685268DA62EA
:1021D0007047024B4FF0FF32DA627047EC03002089
:1021E00010B50446006B00F067FD204600F064FD6A
:1021F00010BD2DE9F04780469946089D099F0A9C2D
:10220000266B02F18042013A06EB820626F00706B1
:1022100000230F2B07D8C85CE21882F83400CA5C90
:102220000AB10133F5E7002384F84330062D00D9C5
:102230000625E56265644FF0000AC4F848A0201D39
:10224000FFF780FF04F11800FFF77CFF2461C5F160
:102250000705A5616462C4F84CA084F850A04A4602
:102260004146304600F020FB206007B13C60BDE8ED
:10227000F087000070B5002407E004EB84029300AF
:1022800010481844FFF753FF0134062CF5D90E4CC3
:1022900004F1BC063046FFF74AFF04F1D00528469A
:1022A000FFF745FF04F11400FFF741FF04F1E400DC
:1022B000FFF73DFF2046FFF73AFFA662C4F8F8504B
:1022C00070BD00BF1C040020EC03002038B505469B
:1022D00000F018FB264BD3F8FC200132C3F8FC2099
:1022E000D3F8003173B1224BD3F804318BB9204BB2
:1022F000D3F80031DA6AEB6A9A420AD81C4BC3F869
:10230000005106E01A4BC3F80051D3F8FC30012B02
:102310002AD0174CD4F808310133C4F80831EB6ADD
:1023200001229A40D4F80C110A43C4F80C2104F19C
:10233000300003EB83039A00291D1044FFF705FFCB
:1023400000F002FBD4F804316BB1D4F80031DA6A42
:10235000EB6A9A4207D2074B4FF080521A60BFF3E4
:102360004F8FBFF36F8F38BDFFF784FFD1E700BFFA
:10237000EC03002004ED00E070B504460E461F4B50
:10238000D3F81051D3F800010430FFF704FF60B90F
:102390001A4BD3F80021D16A012202FA01F1D3F8D5
:1023A0000C2122EA0102C3F80C21B4F1FF3F12D044
:1023B0002C44124BD3F800315C60A54214D80F4D69
:1023C000A86AD5F800110431FFF7CBFEEB6AA342EF
:1023D00012D9EC6210E0002EEAD00848D0F80011C3
:1023E0000431FFF7B2FE07E0044BD3F8F800D3F84E
:1023F00000110431FFF7B5FE70BD00BFEC030020F3
:102400002DE9F04385B00746884615469946900069
:1024100000F0D8FBF8B10646542000F0D3FB044688
:10242000A8B10663D4B10023039302940D9B0193DA
:102430000C9B00934B462A4641463846FFF7D9FE8F
:102440002046FFF743FF012005B0BDE8F08330468A
:1024500000F032FCE6E74FF0FF30F5E74FF0FF30D9
:10246000F2E7000000B583B0174B019300230093FF
:10247000802216491648FFF7C3FF012805D0B0F1A6
:10248000FF3F17D003B05DF804FB4FF0500383F318
:102490001188BFF36F8FBFF34F8F0E4B4FF0FF329A
:1024A000DA620122C3F804210022C3F8102100F0EF
:1024B000C5FAE7E74FF0500383F31188BFF36F8F3E
:1024C000BFF34F8FFEE700BF08050020403E000825
:1024D00089270008EC030020034AD2F818310133A1
:1024E000C2F81831704700BFEC0300202DE9F0411D
:1024F000404BD3F81831002B6CD13E4BD3F8105120
:102500000135C3F81051CDB99B6A1B6843B14FF038
:10251000500383F31188BFF36F8FBFF34F8FFEE734
:10252000344B9A6AD3F8F8109962C3F8F820D3F8BC
:1025300020210132C3F82021FFF740FE2D4BDB6A3A
:10254000AB423DD900242B4AD2F80031DB6A03EBC1
:10255000830399000A44136B012B42D9012440E004
:102560000124244B9B6A1B6863B3224B9B6ADB6884
:10257000DE6873689D422AD306F104084046FFF7DF
:102580000AFEB36A1BB106F11800FFF704FEF36AF6
:1025900001229A40174FD7F80C110A43C7F80C21B3
:1025A00007F1300003EB83039A0041461044FFF724
:1025B000CCFDF26AD7F80031DB6A9A42D0D2D0E77C
:1025C0000024CEE70B4B4FF0FF32DA62BBE7094A3B
:1025D000D362B8E7074AD2F824310133C2F8243174
:1025E0000024044BD3F8283103B101242046BDE870
:1025F000F08100BFEC030020394BD3F8183143B908
:102600004FF0500383F31188BFF36F8FBFF34F8FE9
:10261000FEE770B500F076F9314BD3F81821013A96
:10262000C3F81821D3F81831002B54D12C4BD3F810
:10263000FC3023B9002400F087F9204670BD002447
:10264000274B5B692BB3264D2B6ADC6804F118001D
:10265000FFF7A1FD261D3046FFF79DFDE36A01222D
:102660009A40D5F80C110A43C5F80C2105F1300049
:1026700003EB83039A0031461044FFF766FDE26ADC
:10268000D5F80031DB6A9A42DAD30122C5F8282155
:10269000D6E70CB1FFF792FD114BD3F8244164B19A
:1026A000FFF724FF18B10E4B0122C3F82821013C8B
:1026B000F6D10B4B0022C3F82421094BD3F8283163
:1026C0005BB1084B4FF080521A60BFF34F8FBFF3DE
:1026D0006F8F0124AFE70024ADE70024ABE700BF14
:1026E000EC03002004ED00E010B5B0B104460F4B40
:1026F000D3F8183143B14FF0500383F31188BFF37F
:102700006F8FBFF34F8FFEE7FFF7E6FE00212046F5
:10271000FFF732FEFFF770FF38B9054B4FF08052DC
:102720001A60BFF34F8FBFF36F8F10BDEC03002013
:1027300004ED00E038B5134BD3F814310BB3FFF7B9
:10274000CBFE104BD3F8E440FFF756FF002CF2D03D
:1027500000F0D8F80B4CD4F8F030DD68281DFFF7F6
:102760001AFDD4F8FC30013BC4F8FC30D4F8143125
:10277000013BC4F8143100F0E7F82846FFF730FDBC
:10278000D9E738BDEC03002008B5FFF7D3FF064BAF
:102790001B6B012BF9D9054B4FF080521A60BFF328
:1027A0004F8FBFF36F8FF0E7EC03002004ED00E0E4
:1027B000224BD3F8183123B1204B0122C3F8282132
:1027C00070471E4A0023C2F82831D2F80C31B3FA00
:1027D00083F3DBB2C3F11F0303EB830081000A44E0
:1027E000126B42B94FF0500383F31188BFF36F8F20
:1027F000BFF34F8FFEE710B4104A9900CC18A00029
:102800001044446B646844633032194488000830D3
:10281000024494420BD0094903EB83039A000A4413
:10282000536BDB68C1F800315DF8044B7047616899
:102830000248142202FB03025163ECE7EC03002080
:102840000B4B1B68B3F1FF3F08D04FF0500383F3ED
:102850001188BFF36F8FBFF34F8FFEE74FF0500328
:1028600083F31188BFF36F8FBFF34F8FFEE700BF75
:102870000800002006480068006880F3088862B6F7
:1028800061B6BFF34F8FBFF36F8F00DF00BF000053
:1028900008ED00E0DFF80C00016841F47001016010
:1028A0007047000088ED00E04FF0807340F8043C72
:1028B00021F0010140F8081C054B40F80C3C40F8A1
:1028C000202C6FF0020340F8243C4438704700BFCE
:1028D0004128000800000000000000000000000087
:1028E000074B19680868B0E8F04F80F30988BFF318
:1028F0006F8F4FF0000080F311887047AFF30080B6
:10290000EC0400204FF0500383F31188BFF36F8F66
:10291000BFF34F8F0A4A136801331360012B00D0B5
:102920007047084B1B6813F0FF0FF9D04FF05003AE
:1029300083F31188BFF36F8FBFF34F8FFEE700BFA4
:102940000800002004ED00E0094B1B6843B94FF07C
:10295000500383F31188BFF36F8FBFF34F8FFEE7F0
:10296000013B034A13600BB983F31188704700BF22
:10297000080000200000000000000000000000002F
:10298000EFF30980BFF36F8F154B1A681EF0100F1D
:1029900008BF20ED108A20E9F04F10604DF8043D8B
:1029A0004FF0500080F31188BFF34F8FBFF36F8F4C
:1029B000FFF7FEFE4FF0000080F3118808BC196895
:1029C0000868B0E8F04F1EF0100F08BFB0EC108A96
:1029D00080F30988BFF36F8F704700BFAFF30080AB
:1029E000EC04002008B54FF0500383F31188BFF3C7
:1029F0006F8FBFF34F8FFFF779FD18B1034B4FF087
:102A000080521A60002383F3118808BD04ED00E0B2
:102A1000064B1B68064AA2FB03239B09013B054AA0
:102A20001360054B07221A60704700BFCC030020DB
:102A3000D34D621014E000E010E000E0314B1A6862
:102A4000314B9A420DD02F4B1A68304B9A4211D11C
:102A50004FF0500383F31188BFF36F8FBFF34F8F95
:102A6000FEE74FF0500383F31188BFF36F8FBFF37E
:102A70004F8FFEE700B583B0254B1A78D2B2019292
:102A8000FF221A701B78DBB28DF803309DF80330FB
:102A900003F050031F4A1370072353609DF803305F
:102AA00013F0800F0AD01B4A5368013B53609DF816
:102AB00003305B00DBB28DF80330EFE7154A536853
:102AC0001B0203F4E0635360019BDBB2104A1370F6
:102AD000114B1A6842F470021A601A6842F0704290
:102AE0001A60FFF795FF0D4B00221A60FFF7D2FE28
:102AF0000B4A136843F040431360FFF7BBFEFFF738
:102B00009FFE00BF00ED00E071C20F4170C20F4197
:102B100000E400E01805002020ED00E0080000209F
:102B200034EF00E0104A12F0070F1AD0D11D21F047
:102B30000701C1F5705313440A460C490A6000208E
:102B400048601344083B23F007038B60586018600B
:102B5000981A50601360C86008614FF000434B61E1
:102B600070474FF47053E8E7380500202005002037
:102B700010B4134B1A6882421BD359685C18844204
:102B800003D1406801445960184641684418A24284
:102B900013D10B4CA468A2420DD05268114441607D
:102BA0001A6812680260984200D018605DF8044B01
:102BB00070471346DEE70460F5E70260F3E700BF05
:102BC0002005002070B50446FFF786FC394B9B6852
:102BD000BBB1384B5B691C4262D1ACB1083414F014
:102BE000070F11D024F00704083404F007035BB189
:102BF0004FF0500383F31188BFF36F8FBFF34F8FF4
:102C0000FEE7FFF78FFFE4E7002C4BD0294B1B6951
:102C1000A34249D3274B1D6801E02B4615466A683D
:102C2000A24202D22A68002AF7D1224A9268AA4216
:102C30003CD01E6808362A681A606B681B1B102B74
:102C400010D9281910F0070F08D04FF0500383F364
:102C50001188BFF36F8FBFF34F8FFEE743606C6047
:102C6000FFF786FF6968134A13695B1A1361D2681C
:102C7000934201D20F4AD3600E4B5B690B436B60EA
:102C800000232B60FFF7B8FC16F0070F10D04FF0B1
:102C9000500383F31188BFF36F8FBFF34F8FFEE7AD
:102CA0000026EFE70026EDE70026EBE70026E9E740
:102CB000304670BD2005002080B338B50446A0F131
:102CC000080550F8042C164949690A4208D14FF00A
:102CD000500383F31188BFF36F8FBFF34F8FFEE76D
:102CE00050F8080C40B14FF0500383F31188BFF344
:102CF0006F8FBFF34F8FFEE722EA010244F8042CE6
:102D0000FFF7EAFB54F8041C054A13690B441361EE
:102D10002846FFF72DFFFFF76FFC38BD704700BF57
:102D20002005002000B589B00291013809280BD890
:102D3000DFE800F0050D131920262C32393F082258
:102D400001A91F48FFF72CF909B05DF804FB0C221C
:102D500001A91B48FFF724F9F6E7002201A9194849
:102D6000FFF71EF9F0E704220DEB02011548FFF70B
:102D700017F9E9E7082201A91248FFF711F9E3E77B
:102D80000C2201A90F48FFF70BF9DDE7002201A98A
:102D90000D48FFF705F9D7E704220DEB02010A48B9
:102DA000FFF7FEF8D0E7082201A90748FFF7F8F877
:102DB000CAE70C2201A90448FFF7F2F8C4E700BFF4
:102DC000B843002004430020C842002008B5013861
:102DD00009280BD8DFE800F0050B11171D242B3153
:102DE000373E002204211F48FDF754FE08BD002293
:102DF00008211C48FDF74EFEF8E7002240211A4842
:102E0000FDF748FEF2E7002280211748FDF742FE59
:102E1000ECE700224FF480711348FDF73BFEE5E735
:102E200000224FF400711048FDF734FEDEE7002267
:102E300040210E48FDF72EFED8E7002280210B48E6
:102E4000FDF728FED2E700224FF480710748FDF716
:102E500021FECBE700224FF400710448FDF71AFE73
:102E6000C4E700BF00000240000802400004024026
:102E700008B5013809280BD8DFE800F0050B111759
:102E80001D242B31373E012204211F48FDF702FE8D
:102E900008BD012208211C48FDF7FCFDF8E70122CE
:102EA00040211A48FDF7F6FDF2E70122802117487C
:102EB000FDF7F0FDECE701224FF480711348FDF7B8
:102EC000E9FDE5E701224FF400711048FDF7E2FD4E
:102ED000DEE7012240210E48FDF7DCFDD8E70122A4
:102EE00080210B48FDF7D6FDD2E701224FF4807117
:102EF0000748FDF7CFFDCBE701224FF400710448EE
:102F0000FDF7C8FDC4E700BF000002400008024012
:102F100000040240642303FB00F3074880FB032006
:102F200018444011C0EB4013C3EB831300EBC30004
:102F30004300581E80B2704789888888F0B585B0F4
:102F40000E46174604AA02F8040D094C4FF47A7590
:102F500000950123D0212046FEF72CF80095BBB246
:102F60003246D0212046FEF7E7F805B0F0BD00BF9D
:102F70008C410020B0B582B002AF1346083222F077
:102F80000702ADEB020D02AA15468DF808000020DD
:102F900003E00C18013024782C549842F9DB0133FB
:102FA0004FF47A7100919BB2D0210248FEF702F8EB
:102FB000BD46B0BD8C41002000B583B0012201A9FF
:102FC0000220FFF7BBFF9DF804100B0903EB8303FE
:102FD0005A00CA4214BF0120002003B05DF804FB70
:102FE00000B583B0012201A90320FFF7A7FF9DF8D8
:102FF0000400003018BF012003B05DF804FB10B5D9
:1030000082B00446072269460120FFF797FF9DF82A
:103010000030003318BF012323709DF801100B0905
:1030200003EB83035A001346CA4214BF0123002353
:1030300063709DF80230003318BF0123A3709DF820
:103040000430003318BF0123E3709DF805300033CE
:1030500018BF012323719DF806100B0903EB8303AE
:103060005A001346CA4214BF01230023637102B001
:1030700010BD00B583B002A9402301F8043D012230
:103080000C20FFF777FF03B05DF804FB0A3801441A
:103090000139024B13F82100704700BF0C000020DB
:1030A00000B585B000230093019302930393144865
:1030B000144A02604FF4803242608360036183618E
:1030C0000362C362104A8262C3600122C261036369
:1030D0004261FDF7C9FA68B90923009301230193FE
:1030E0000023029369460648FDF7E8FA28B905B0BF
:1030F0005DF804FB00F078FAEEE700F075FAF6E709
:1031000040410020002001400100000F00B589B0BF
:10311000002303930493059306930793026803F136
:10312000804303F590339A4202D009B05DF804FB66
:103130000021019103F58C335A6C42F480725A6479
:103140005A6C02F480720192019A02911A6B42F059
:1031500002021A631B6B03F002030293029B022319
:1031600003930323049303A90148FDF7C1FBDCE7A4
:103170000004024070B52CE02046FFF779FE0134D0
:103180000A2C22DC2946E0B2FFF780FF022807D094
:1031900003280AD00128EFD02046FFF717FEEEE7FC
:1031A00031462046FFF7BEFDE9E7114B1B78012BA6
:1031B00007D0C6F5F441113189B22046FFF7B2FDC0
:1031C000DDE72046FFF702FED9E74EF66020FEF766
:1031D000A5FFFFF705FF054610B9054B00221A7041
:1031E000FFF7EAFEFFF796FE06460124C8E700BF98
:1031F00038410020884200D870470846FCE70000AC
:10320000F0B585B002A8FFF7FAFEFFF732FF684677
:10321000FFF7F5FE00262BE029462046FFF782FD4A
:1032200001340A2C1EDC9DF80210E0B2FFF72EFFDD
:10323000022807D003280ED00128EDD02046FFF742
:10324000C5FDEDE729463846FFF7D4FF0146204685
:10325000FFF768FDE4E7114B01221A702046FFF7E3
:10326000B5FDDDE74EF66020FEF758FF0136F6B2F9
:10327000092E10D8FFF7A0FEFFF74CFE0746731C7F
:103280004FF0FF3595FBF3F547F6122313FA85F55A
:10329000ADB20124C5E705B0F0BD00BF3841002044
:1032A00030B587B0FFF7ACFF01AC064D0FCD0FC4B2
:1032B0002B682360002101A8FEF716FF024B18605F
:1032C00007B030BD143E0008884100202DE9F043CE
:1032D0008BB00024059406940794089409940094F4
:1032E0004F4B1A6B42F004021A631A6B02F004028D
:1032F0000092009A01941A6B42F080021A631A6BD2
:1033000002F080020192019A02941A6B42F00102CB
:103310001A631A6B02F001020292029A03941A6B6A
:1033200042F002021A631A6B02F002020392039A3D
:1033300004941A6B42F008021A631B6B03F0080333
:103340000493049BDFF8E490224644F2300148469F
:10335000FDF7A0FB334E224601213046FDF79AFBD4
:10336000DFF8CC80224605214046FDF793FB4BF663
:103370000F43059303250695079405A94846FDF7D5
:10338000B7FA44F23003059301270697079408948F
:1033900005A94846FDF7ACFA0597069707940894E7
:1033A00005A93046FDF7A4FA05230593069707946F
:1033B000089405A94046FDF79BFA4FF220030593B8
:1033C0000695079405A94046FDF792FA4FF400735D
:1033D00005930694079405A93046FDF789FA4FF442
:1033E000E053059302230693079408950A23099353
:1033F00005A93046FDF77CFA4FF400430593069586
:10340000079405A93046FDF773FA04230593069542
:10341000079405A90448FDF76BFA0BB0BDE8F083EB
:103420000038024000000240000C02400008024048
:103430000004024008B50B480B4B03600B4B436084
:1034400000238360C3604FF4804202614361836163
:10345000C3610362FDF720FD00B908BD00F0C4F8A8
:10346000FBE700BFE041002000580040A0860100BB
:1034700008B50B480B4B03604CF2503343600023FC
:103480008360C3604FF48042026143618361C36122
:103490000362FDF701FD00B908BD00F0A5F8FBE7E8
:1034A0008C410020005C00402DE9F0438BB00023EC
:1034B0000593069307930893099303683F4A934241
:1034C00005D03F4A93423AD00BB0BDE8F0830025C7
:1034D00000953C4C236B43F002032363236B03F002
:1034E00002030093009B4FF4806305934FF0120991
:1034F000CDF818904FF00108CDF81C8003270897ED
:1035000004230993304E05A93046FDF7F1F908234D
:103510000593CDF81890CDF81C80089709230993DE
:1035200005A93046FDF7E4F90195236C43F48003C7
:103530002364236C03F480030193019BC4E70025FB
:103540000295204C236B43F001032363236B03F0AC
:1035500001030293029B0395236B43F00203236351
:10356000236B03F002030393039B4FF480730593D3
:103570004FF01208CDF81880012707970326089608
:103580000423099305A91148FDF7B2F91023059307
:10359000CDF81880079708960923099305A90A48CA
:1035A000FDF7A6F90495236C43F400032364236C10
:1035B00003F400030493049B86E700BF0058004017
:1035C000005C00400038024000040240000002405D
:1035D00008B50268034B9A4200D008BDFCF79AFF79
:1035E000FBE700BF000C0040FEE7000000B595B00F
:1035F0003022002108A800F0F9FB00230393049374
:103600000593069307930193214A116C41F0805171
:103610001164126C02F080520192019A02931D4AC9
:10362000136823F4404343F400431360136803F426
:1036300040430293029B012308934FF48033099384
:1036400002230E934FF480030F93192310934FF42A
:10365000A8731193042312930723139308A8FDF76B
:10366000DFFE80B90F230393022104910023059309
:103670004FF480520692079303A8FEF7F1F820B9A1
:1036800015B05DF804FBFFF7AFFFFFF7ADFF00BF1C
:10369000003802400070004008B5FCF721FFFFF73A
:1036A000A5FFFFF713FE00F051FB00F0F3FA00F066
:1036B00095FAFFF7DDFEFFF7BDFE00F00DF800F014
:1036C0002DF900F0F5F8FFF7EBFC00F035FAFFF705
:1036D000E7FDFEF704FDFEE708B50D480D4B03605E
:1036E0004FF48273436000238360C36003614361CE
:1036F0004FF480228261C3610362436283620A23C2
:10370000C362FEF78DF900B908BDFFF76DFFFBE757
:10371000344200200030014000B589B000230393FB
:1037200004930593069307930268154B9A4202D0BF
:1037300009B05DF804FB0021019103F584335A6C54
:1037400042F480525A645A6C02F480520192019AF7
:1037500002911A6B42F001021A631B6B03F0010322
:103760000293029BF0230393022304930323069303
:103770000523079303A90348FDF7BAF8D8E700BF6C
:10378000003001400000024000B583B000220092EA
:103790000D4B596C41F480415964596C01F48041DE
:1037A000009100990192196C41F0805119641B6CD1
:1037B00003F080530193019B0F216FF00100FDF78F
:1037C00057F803B05DF804FB0038024010B588B02C
:1037D000002201463220FDF74BF83220FDF77CF83D
:1037E00000240194144B1A6C42F008021A641B6CFA
:1037F00003F008030193019B02A903A8FEF7F2F866
:10380000FEF7E0F843000D48A0FB03239B0C013BAF
:103810000B480C4A026040F2E732C2604360046128
:103820008460FEF75DFB10B1012008B010BD0448B4
:10383000FEF71FFAF9E700BF0038024083DE1B43A2
:103840008C420020000C00407047FEE7FEE7FEE7D8
:10385000FEE7704708B50248FEF73BFA08BD00BF17
:103860008C4200200F49D1F8883043F47003C1F82E
:1038700088300D4B1A6842F001021A6000209860EF
:103880001A6822F0847222F480321A60074A5A6061
:103890001A6822F480221A60D8604FF000638B60AF
:1038A000704700BF00ED00E00038024010300024F7
:1038B00000B589B0002303930493059306930793FF
:1038C000019302931348144A026043608360C3600B
:1038D00003614361FEF704FB98B9072303930023B8
:1038E000049303A90B48FEF7D0F968B900230193AC
:1038F000029301A90748FEF7C1FB40B909B05DF882
:1039000004FBFFF771FEE8E7FFF76EFEEEE7FFF757
:103910006BFEF3E7404300200000014000B58DB08E
:1039200000230793089309930A930B930093019341
:10393000029303930493059306931848184A026070
:1039400043608360C3600361FEF7CAFAC8B91348D5
:10395000FEF7DFFAC0B900230793089307A90F48C1
:10396000FEF793F998B96023009300220192029226
:10397000049269460948FEF713FB58B90DB05DF88B
:1039800004FBFFF731FEE2E7FFF72EFEE3E7FFF768
:103990002BFEE8E7FFF728FEF0E700BF7C4300209E
:1039A0000040014082B00368104A934204D0104A9C
:1039B00093420ED002B07047002300930D4B5A6C17
:1039C00042F001025A645B6C03F001030093009B18
:1039D000F0E700230193074B5A6C42F480325A649B
:1039E0005B6C03F480330193019BE3E7000001402B
:1039F000004001400038024084B00368B3F1804FBA
:103A000007D0174A934211D0164A93421BD004B0F4
:103A1000704700230193144B1A6C42F001021A64A0
:103A20001B6C03F001030193019BF0E70023029359
:103A30000D4B1A6C42F002021A641B6C03F0020375
:103A40000293029BE3E700230393074B1A6C42F0B7
:103A500004021A641B6C03F004030393039BD6E770
:103A600000040040000800400038024000B589B062
:103A70000023039304930593069307930368B3F11C
:103A8000804F08D0264A93421CD0264A934230D019
:103A900009B05DF804FB00230093234B1A6B42F03E
:103AA00001021A631B6B03F001030093009B0E23BA
:103AB0000393022304930123079303A91B48FCF7F4
:103AC00017FFE5E700230193174B1A6B42F004023E
:103AD0001A631B6B03F004030193019B4FF4707393
:103AE000039302230493079303A91148FCF700FFF3
:103AF000CEE7002302930C4B1A6B42F002021A63CA
:103B00001B6B03F002030293029B4FF47073039349
:103B100002230493079303A90648FCF7E9FEB7E7DD
:103B2000000400400008004000380240000002404D
:103B3000000802400004024000B58BB00023089347
:103B400009930193029303930493059306930793B8
:103B500021484FF08042026007224260836047F6AE
:103B60001122C2600361FEF7D4F930BB0023089331
:103B7000099308A91848FEF781FA08BB602301934E
:103B8000002302930393059304220DEB02011248D4
:103B9000FEF706FAB8B9082201A90F48FEF700FAA5
:103BA000A0B90C2201A90C48FEF7FAF988B90A4815
:103BB000FFF75CFF0BB05DF804FBFFF715FDD5E7E1
:103BC000FFF712FDDAE7FFF70FFDE4E7FFF70CFD63
:103BD000E7E7FFF709FDEAE7B843002000B58BB03F
:103BE000002308930993019302930393049305938D
:103BF000069307932548264A0260072242608360A5
:103C000047F61122C2600361FEF783F958BB002317
:103C10000893099308A91D48FEF730FA30BB6023CA
:103C20000193002202920392059201A91748FEF720
:103C3000B7F9F0B904220DEB02011448FEF7B0F910
:103C4000D0B9082201A91148FEF7AAF9B8B90C2287
:103C500001A90E48FEF7A4F9A0B90C48FFF706FF2A
:103C60000BB05DF804FBFFF7BFFCD0E7FFF7BCFC2F
:103C7000D5E7FFF7B9FCDDE7FFF7B6FCE1E7FFF7B3
:103C8000B3FCE4E7FFF7B0FCE7E700BF0443002024
:103C90000004004000B58BB0002308930993019302
:103CA0000293039304930593069307932548264AAA
:103CB000026007224260836047F61122C2600361FE
:103CC000FEF727F958BB00230893099308A91D485C
:103CD000FEF7D4F930BB60230193002202920392D5
:103CE000059201A91748FEF75BF9F0B904220DEB24
:103CF00002011448FEF754F9D0B9082201A911486D
:103D0000FEF74EF9B8B90C2201A90E48FEF748F9A2
:103D1000A0B90C48FFF7AAFE0BB05DF804FBFFF753
:103D200063FCD0E7FFF760FCD5E7FFF75DFCDDE75C
:103D3000FFF75AFCE1E7FFF757FCE4E7FFF754FC15
:103D4000E7E700BFC84200200008004070470000BD
:103D5000DFF834D0002103E00C4B5B5843500431B2
:103D60000B480C4B42189A42F6D30B4A02E0002350
:103D700042F8043B094B9A42F9D3FFF773FD00F078
:103D800011F8FFF789FC704700000120603E000831
:103D900000000020D0030020D0030020F4430020C6
:103DA000FEE7000070B50D4E0D4CA41BA4100025BD
:103DB000A54209D10B4E0C4C00F020F8A41BA41016
:103DC0000025A54205D170BD56F82530984701352C
:103DD000EEE756F8253098470135F2E7583E0008DF
:103DE000583E0008583E00085C3E00080244034666
:103DF000934200D1704703F8011BF9E7F8B500BF03
:103E0000F8BC08BC9E467047F8B500BFF8BC08BCBB
:043E10009E46704713
:103E1400483E000875310008000000000000000062
:103E24008000000000000000000000000102030404
:103E340006070809000000000102030449444C4538
:0C3E44000000000054696D657200000071
:083E5000C0C3FF7F0100000068
:043E5800C501000898
:043E5C00A1010008B8
:103E60000100000010000000AAAAAAAA0000000099
:103E70000000000000000000000000000000000042
:103E80000000000000000000000000000200000030
:103E9000010000000100000001000000010000001E
:103EA000010000000100000001000000010000000E
:103EB00001000000010000000100000001000000FE
:103EC00001000000030000000000000000000000EE
:103ED00000000000000000000000000000000000E2
:103EE00000000000000000000000000002000000D0
:103EF00001000000010000000100000001000000BE
:103F000001000000010000000100000001000000AD
:103F1000010000000100000001000000010000009D
:103F2000010000000300000000000000000000008D
:103F30000000000000000000000000000000000081
:103F40000000000000000000000000000000000071
:103F5000020000000100000001000000010000005C
:103F6000010000000100000001000000010000004D
:103F7000010000000100000001000000010000003D
:103F8000030000000000000000000000000000002E
:103F90000000000000000000000000000000000021
:103FA0000000000000000000000000000000000011
:103FB00000000000020000000100000001000000FD
:103FC00001000000010000000100000001000000ED
:103FD00001000000010000000100000001000000DD
:103FE00003000000000000000000000000000000CE
:103FF00000000000000000000000000000000000C1
:1040000000000000000000000000000000000000B0
:10401000000000000200000001000000010000009C
:10402000010000000100000001000000010000008C
:10403000010000000100000001000000010000007C
:10404000030000000000000000000000000000006D
:104050000000000000000000000000000000000060
:104060000000000000000000000000000000000050
:10407000000000000000000000000000020000003E
:10408000010000000100000001000000010000002C
:10409000010000000100000001000000010000001C
:1040A000010000000300000000000000000000000C
:1040B0000000000000000000000000000000000000
:1040C00000000000000000000000000000000000F0
:1040D00000000000000000000000000000000000E0
:1040E00000000000000000000000000000000000D0
:1040F00000000000000000000000000000000000C0
:1041000000000000000000000000000000000000AF
:10411000000000000000000000000000000000009F
:10412000000000000000000000000000000000008F
:10413000000000000000000000000000000000007F
:10414000000000000000000000000000000000006F
:10415000000000000000000000000000000000005F
:10416000000000000000000000000000000000004F
:10417000000000000000000000000000000000003F
:10418000000000000000000000000000000000002F
:10419000000000000000000000000000000000001F
:1041A000000000000000000000000000000000000F
:1041B00000000000000000000000000000000000FF
:1041C00000000000000000000000000000000000EF
:1041D00000000000000000000000000000000000DF
:1041E00000000000000000000000000000000000CF
:1041F00000000000000000000000000000000000BF
:1042000000000000000000000000000000000000AE
:10421000000000000000000000000000000000009E
:104220000000000000000000000000000024F40076
:0400000508003D5161
:00000001FF
